:10000000020D5F00438701220212EB02113EC2C5BE
:0F0010007F051210CDE4900331F02275C13F221D
:1000230002104FE709F608DFFA8046E709F208DF16
:10003300FA803E88828C83E709F0A3DFFA8032E3FB
:1000430009F608DFFA8078E309F208DFFA8070889E
:10005300828C83E309F0A3DFFA806489828A83E0D8
:10006300A3F608DFFA805889828A83E0A3F208DFC7
:10007300FA804C80D280FA80C680D4806980F28076
:1000830033801080A680EA809A80A880DA80E2809C
:10009300CA803389828A83ECFAE493A3C8C582C8F1
:1000A300CCC583CCF0A3C8C582C8CCC583CCDFE95B
:1000B300DEE7800D89828A83E493A3F608DFF9ECF7
:1000C300FAA9F0EDFB2289828A83ECFAE0A3C8C582
:1000D30082C8CCC583CCF0A3C8C582C8CCC583CCA9
:1000E300DFEADEE880DB89828A83E493A3F208DF18
:1000F300F980CC88F0EF60010E4E60C388F0ED24E8
:1001030002B4040050B9F582EB2402B4040050AFEA
:10011300232345822390007673BB010689828A8359
:10012300E0225002E722BBFE02E32289828A83E4B3
:100133009322BB010CE58229F582E5833AF583E03E
:10014300225006E92582F8E622BBFE06E92582F85D
:10015300E222E58229F582E5833AF583E49322BB23
:10016300010689828A83F0225002F722BBFE01F343
:1001730022F8BB010DE58229F582E5833AF583E890
:10018300F0225006E92582C8F622BBFE05E9258246
:10019300C8F222BC000BBE0029EF8DF084FFADF046
:1001A30022E4CCF875F008EF2FFFEE33FEEC33FCBE
:1001B300EE9DEC984005FCEE9DFE0FD5F0E9E4CEF4
:1001C300FD22EDF8F5F0EE8420D21CFEADF075F0C3
:1001D30008EF2FFFED33FD4007985006D5F0F222CC
:1001E300C398FD0FD5F0EA22C2D5EC30E709B2D5AA
:1001F300E4C39DFDE49CFCEE30E715B2D5E4C39F58
:10020300FFE49EFE120196C3E49DFDE49CFC800383
:1002130012019630D507C3E49FFFE49EFE22C5F08A
:10022300F8A3E028F0C5F0F8E58215827002158383
:10023300E038F022BB010A89828A83E0F5F0A3E06B
:1002430022500687F009E71922BBFE07E3F5F00900
:10025300E3192289828A83E493F5F074019322BB24
:10026300010A89828A83F0E5F0A3F0225006F70998
:10027300A7F01922BBFE06F3E5F009F31922E88F74
:10028300F0A4CC8BF0A42CFCE98EF0A42CFC8AF017
:10029300EDA42CFCEA8EF0A4CDA8F08BF0A42DCC19
:1002A3003825F0FDE98FF0A42CCD35F0FCEB8EF072
:1002B300A4FEA9F0EB8FF0A4CFC5F02ECD39FEE458
:1002C3003CFCEAA42DCE35F0FDE43CFC2275F0089D
:1002D300758200EF2FFFEE33FECD33CDCC33CCC58B
:1002E3008233C5829BED9AEC99E58298400CF582A6
:1002F300EE9BFEED9AFDEC99FC0FD5F0D6E4CEFB18
:10030300E4CDFAE4CCF9A88222B800C1B90059BA05
:10031300002DEC8BF084CFCECDFCE5F0CBF9781833
:10032300EF2FFFEE33FEED33FDEC33FCEB33FB102D
:10033300D703994004EB99FB0FD8E5E4F9FA227847
:1003430018EF2FFFEE33FEED33FDEC33FCC933C959
:1003530010D7059BE99A4007EC9BFCE99AF90FD863
:10036300E0E4C9FAE4CCFB2275F010EF2FFFEE3383
:10037300FEED33FDCC33CCC833C810D7079BEC9AC2
:10038300E899400AED9BFDEC9AFCE899F80FD5F04B
:10039300DAE4CDFBE4CCFAE4C8F922EB9FF5F0EA0A
:1003A3009E42F0E99D42F0EC6480C864809845F079
:1003B30022EB9FF5F0EA9E42F0E99D42F0E89C456E
:1003C300F022E8600FECC313FCED13FDEE13FEEF18
:1003D30013FFD8F122BB010789828A830205A75044
:1003E30005E9F802059BBBFE05E9F80205B389821E
:1003F3008A830205BFBB010789828A830204965060
:1004030005E9F802067ABBFE05E9F802068622BB77
:10041300010DE58229F582E5833AF58302049650BE
:1004230007E92582F802067ABBFE07E92582F8026E
:10043300068622BB010DE58229F582E5833AF58321
:1004430002062E5007E92582F802060EBBFE07E9D5
:100453002582F8020663E58229F582E5833AF5836E
:100463000205BFBB010DE58229F582E5833AF583D9
:100473000205DC5007E92582F80205CFBBFE07E938
:100483002582F80205E8E58229F582E5833AF583BA
:100493000205F5ECF0A3EDF0A3EEF0A3EFF022A834
:1004A300828583F0D083D0821204B91204B9120476
:1004B300B91204B9E473E493A3C583C5F0C583C833
:1004C300C582C8F0A3C583C5F0C583C8C582C82249
:1004D300A42582F582E5F03583F58322BB010DE582
:1004E3008229F582E5833AF5830206A45007E925BC
:1004F30082F8020692BBFE07E92582F80206B6E5FA
:100503008229F582E5833AF5830206C8BB0120E51B
:100513008229F582E5833AF583D0F0D0E0F8D0E084
:10052300F9D0E0FAD0E0FBE8C0E0C0F00206AD503D
:1005330018E92582F8D083D082D0E0F9D0E0FAD050
:10054300E0FBC082C08302069BBBFE18E92582F84C
:10055300D083D082D0E0F9D0E0FAD0E0FBC082C0F3
:10056300830206BF228A838982E473EC8EF0A4CCD3
:10057300C5F0CCCDF8EFA4CEC5F02DFDE43CFCE8EE
:10058300A42EC8C5F03DFDE43CFCEFA4FFE5F02834
:10059300FEE43DFDE43CFC22E6FC08E6FD08E6FE45
:1005A30008E6FF22E0FCA3E0FDA3E0FEA3E0FF22B8
:1005B300E2FC08E2FD08E2FE08E2FF22E493FC7499
:1005C3000193FD740293FE740393FF22E6FB08E696
:1005D300F908E6FA08E6CBF822E0F8A3E0F9A3E08D
:1005E300FAA3E0FB22E2FB08E2F908E2FA08E2CB15
:1005F300F822E493F8740193F9740293FA74039361
:10060300FB227401FF3395E0FEFDFC080808E62F8A
:10061300FFF618E63EFEF618E63DFDF618E63CFC4E
:10062300F6227401FF3395E0FEFDFCA3A3A3E02FA4
:10063300FFF0E582158270021583E03EFEF0E5824D
:10064300158270021583E03DFDF0E582158270028C
:100653001583E03CFCF0227401FF3395E0FEFDFCC2
:10066300080808E22FFFF218E23EFEF218E23DFD11
:10067300F218E23CFCF222ECF608EDF608EEF6087E
:10068300EFF622ECF208EDF208EEF208EFF222E6C2
:10069300FB08E6FA08E6F922EBF608EAF608E9F6BB
:1006A30022E0FBA3E0FAA3E0F922EBF0A3EAF0A334
:1006B300E9F022E2FB08E2FA08E2F922EBF208EAA7
:1006C300F208E9F222E493FB740193FA740293F9BA
:1006D30022FAE6FB0808E6F925F0F618E6CA3AF628
:1006E30022D083D082F8E4937012740193700DA327
:1006F300A393F8740193F5828883E4737402936877
:1007030060EFA3A3A380DF8B088A09890A8C0B8D72
:100713000CE4F513F514E50D5401FEE48E15850E76
:1007230016AE0DAF0EFCFDFB7A02F9F812030CE4D2
:10073300FB7A02F9F81202818E178F18E516250C41
:10074300FFE515350BFEE4FCFDFB7A02F9F8120315
:100753000CEF04F519E4F511F512AF19EF3395E039
:10076300FEC3E5129FE5119E4003020896E4F50FD0
:10077300F510AE0FAF10E4FCFDFB7A02F9F8D312CB
:1007830003B44036AE11AF127C027D0012056EE554
:10079300182FFFE5173EFEE5102FFFE50F3EFE1273
:1007A300126474002510F5827400350FF583EFF0A1
:1007B3000510E51070BC050F80B8E51245117006F1
:1007C300AE15AF1680047E007F008E0F8F10AE0F24
:1007D300AF10E4FCFDFB7A02F9F8D31203B44040F6
:1007E300AB08AA09A90A851482851383120135FF70
:1007F30074002510F5827400350FF583EFF0E50CD6
:10080300150C7002150B14450B70030080120510B4
:10081300E5107002050F0514E51470B2051380AEE0
:10082300AE11AF127C027D0012056EE50E2FFFE5BF
:100833000D3EFE120F31E4F50FF510AE0FAF10E4CD
:10084300FCFDFB7A02F9F8D31203B4403BAE11AFBF
:10085300127C027D0012056EE5182FFFE5173EFEA0
:10086300E5102FFFE50F3EFE74002510F58274009E
:10087300350FF583E0FD1211CFEF7002FF22051053
:10088300E51070B7050F80B30512E512700205116C
:1008930002075D7F0122750801750902750A01E4EB
:1008A300F50BC3E50B94057480948040030209A4FF
:1008B300AB08AA09A90A12011C700302099490004B
:1008C300067FFF7EFF7DFF7CFF120436E4FBFAF90F
:1008D300F8C312039E5003020994AB08AA09A90A9C
:1008E30090000112013514606B14600A2402600346
:1008F30002098A020990E92406F9E43AFAC003C01E
:1009030002C0011203D8AB08AA09A90A9000021277
:100913000466EF2BFFEE3AFEED39FDEC38FCD00117
:10092300D002D0031203F8AB08AA09A90A90000D5C
:100933001204DFC003C002C001AB08AA09A90A90D0
:10094300000A1204DF89828A83D001D002D0031205
:10095300056C803DAB08AA09A90A90000D1204DFBB
:10096300C003C002C001AB08AA09A90A90000A1279
:1009730004DF89828A83D001D002D00312056CABD5
:1009830008AA09A90A8006AB08AA09A90AE4120160
:1009930062050B7410250AF50AE43509F509020806
:1009A300A522900339E0FCA3E0FDA3E0FEA3E0242D
:1009B30001FFE43EFEE43DFDE43CFC9003391204F8
:1009C30096900337E0146028146064147003020ADD
:1009D30065147003020A7E24046003020A8E9003E6
:1009E300391204A2000000007F02120EE1020A770E
:1009F30090032FE06402705890033DE0FCA3E0FDF8
:100A0300A3E0FEA3E0FF900339E0F8A3E0F9A3E03D
:100A1300FAA3E0FBD31203B440719003391204A28A
:100A2300000000009003377402F0E4FF020EE1902F
:100A3300032FE07056900335E014F0E0D394007474
:100A430080948040167F02120EE19003377403F006
:100A53009003391204A200000000229003377404AB
:100A6300F02290032FE0640270219003391204A254
:100A7300000000009003377401F022C2C17F081206
:100A830010CD7DE87C037F0412128122E51D7003E3
:100A9300020003D3E51C9400748094804040E4F585
:100AA30008C3E5089409748094805032E50875F012
:100AB3000AA42453F582E43402F583C083C0827E02
:100AC30000C3A3E0951CFF0582D58202158315821E
:100AD300E09ED082D083F0A3EFF0050880C3E4F555
:100AE3001DF51CF508C3E508940974809480507CB7
:100AF300E50875F00AA42451F582E43402F583E095
:100B03006065E50875F00AA42453F582E43402F520
:100B13008374FFF5F0120221FED3E5F09400EE6436
:100B23008094805042E50875F00AA42455F582E4C8
:100B33003402F583E0FEA3E0FFE50875F00AA42480
:100B430053F582E43402F583EE8FF012022100E5BF
:100B53000875F00AA42458F582E43402F583A3E06F
:100B6300FAA3E0F91205680508020AE8227DF47C7D
:100B7300017F01121281900337E014603114603D4C
:100B8300147003020C2224036003020C2D9003391A
:100B93001204A20000000090034FE064026003020D
:100BA3000C2D7F02120EE19003377401F0229003A3
:100BB3002FE0640270749003377402F022900339BB
:100BC300E0FCA3E0FDA3E0FEA3E02401FFE43EFE7E
:100BD300E43DFDE43CFC90033912049690034FE09E
:100BE300640170467B14FAF9F8900339E0FCA3E042
:100BF300FDA3E0FEA3E0FF12030C90033D12049655
:100C03007B017A03793D750D00750E047D047C002C
:100C130012070AE4FF120EE19003377403F02290E7
:100C2300032FE0700590033804F022605A0251014B
:100C330001000A000A01FF0899010100640064022F
:100C4300FF1301000101F401F403FF11A2010100EC
:100C530064006406FF001B0101000A000A04FF0C84
:100C6300CA01010001000109FF108F000103E8031D
:100C7300E808FF09A50101003200320AFF0E7500E2
:100C8300010064006405FF12B9011D00011C00414D
:100C9300020000012300022400004103410041033C
:100CA30044004A034500000000000000000000412A
:100CB3000342004103430041034F00041F000000AF
:100CC3000042032B000000AF905307D3EF604E9018
:100CD3000341E06F6008EFF0E4900344F0229003D7
:100CE30044E004F0E0D3940874809480406DEF54A2
:100CF3000364037066F0900342E0FE2445F582E44A
:100D03003403F583EFF0EE2401FFE433FE7C007D32
:100D13000A120196900342EDF07D648037900344FC
:100D2300E0D3940A748094804031E4F0900341E06E
:100D3300FFA3E0FE2445F582E43403F583EFF0EEF0
:100D43002401FFE433FE7C007D0A120196900342E6
:100D5300EDF07DC87C007F0112128122787FE4F6DA
:100D6300D8FD758125020DA60211FAE493A3F8E4D8
:100D730093A34003F68001F208DFF48029E493A3F0
:100D8300F85407240CC8C333C4540F4420C8834009
:100D930004F456800146F6DFE4800B0102040810D8
:100DA300204080900C2EE47E019360BCA3FF543F4F
:100DB30030E509541FFEE493A360010ECF54C02510
:100DC300E060A840B8E493A3FAE493A3F8E493A300
:100DD300C8C582C8CAC583CAF0A3C8C582C8CAC564
:100DE30083CADFE9DEE780BEE4FDFC90025775F0BD
:100DF3000AED1204D3EC75F00AA42583F583E06FA2
:100E0300706190025175F00AED1204D3EC75F00A8B
:100E1300A42583F583E0705990025175F00AED1211
:100E230004D3EC75F00AA42583F5837401F09002D2
:100E33005575F00AED1204D3EC75F00AA42583F579
:100E430083E50DF0A3E50EF0FF90025375F00AED74
:100E53001204D3EC75F00AA42583F583E50DF0A302
:100E6300EFF0220DBD00010CED64094C6003020D8F
:100E7300EE2212117190034FEFF024FD604224C360
:100E8300704A900336E07021A3F090033604F0D249
:100E9300C1E4750EE8750D03F50CF50B7F08120D13
:100EA300EB9003387402F08023E4900336F0C2C160
:100EB30012000E9003387401F07F081210CD800CDD
:100EC300900336E07006A3F0A37403F0900338E0B8
:100ED30024FE6009147003020B70120FC7228F08DF
:100EE300E4F5091212D490032FE0B508037FFE2224
:100EF300D2C5E50824FE600C2402700D9003307403
:100F030001F08005E4900330F0900330E0D36001FA
:100F1300C392C400D2C59003317401F0E4750E325C
:100F2300F50DF50CF50B7F05120DEB7F00228E1AE4
:100F33008F1BE4FCFDFB7A02F9F812030CE4FB7A45
:100F430002F9F8120281E4FFE4FDFC78081203C5FC
:100F53008FC3AE1AAF1BE4FCFDFB7A02F9F8120350
:100F63000CE4FB7A02F9F8120281E48FC475C7809E
:100F730075C50375C65A75C6A500F5C72290032F1C
:100F83007401F0E4900331F0A304F0A37490F0A390
:100F930074FFF0A37403F07B017A037935E4F50D54
:100FA300F50E7D01FC12100DE4900336F0A3F0A3BF
:100FB30004F0FB7A03793D750D00750E047D047C06
:100FC3000002100D90034FE01460122481601B2473
:100FD3007E7036900331E0700E7F028007900331FC
:100FE300E07004FF020EE102000E900335E075F09D
:100FF3000A84E5F0F0E004F07B017A037935E4F547
:101003000DF50E7D01FC12070A228C0B8D0C8B1142
:101013008A128913E4F50FF510C3E510950CE50F5B
:10102300950B5027E50E2510FFE50D350FFE121227
:1010330064AB11AA12A913851082850F83EF1201E5
:10104300740510E51070D2050F80CE22C0E0C08376
:10105300C082C0D075D000C00630992590032BE024
:10106300FEA3E024ABF58274023EF583E06012F543
:101073009990032CE004F0700690032BE004F0C277
:1010830099D006D0D0D082D083D0E032D2A2D2A3DE
:10109300781EE66014900335E075F00A84E5F0905D
:1010A300131793F580C2A38019900335E075F00AF6
:1010B30084FF70047FFF8006EF90131793FF8F80E8
:1010C300C2A2781E06E65401F622E4FDFC90025704
:1010D30075F00AED1204D3EC75F00AA42583F583A9
:1010E300E0B5071690025175F00AED1204D3EC75C2
:1010F300F00AA42583F583E4F0220DBD00010CED75
:1011030064094C70C822E4FFFEE4FDFC000000000B
:1011130000000000000000000000000000000000CC
:10112300000000000DBD00010CBC03E0BDE7DD0FB6
:10113300BF00010EBE03D2BFE7CF22C0E0C0D0750F
:10114300D000C005C006C0077F317EF8E51D6401ED
:101153007002051C751D01AD8AED2FFFE43E8F8AD9
:10116300FF8F8CD007D006D005D0D0D0E0329003CB
:1011730042E0FFA3E0FE6F602174452EF582E43464
:1011830003F583E0FBEE2401FFE433FE7C007D0ADC
:10119300120196900343EDF08002E4FBAF03227843
:1011A30023E66004D2C68016C2C67825E6161870F8
:1011B30001167825E6184670057F031210CD7823B3
:1011C300E67F0070027F017823A60722AB07EEF5C6
:1011D300C3EBF5C48DC275C78075C50275C65A7554
:1011E300C6A500E4F5C7E5C754106410C37001D366
:1011F3007F0040027F0122C2AF1212211211091295
:10120300129D121245120F807DE87C037F0112129A
:10121300811212D4120008D2AF120A8F80FB75BB61
:101223007075B4FF7580FF7591FF7592FF7590FF20
:1012330075A0FF75B0FFE4F5C0C2C5C2C1C2C4C288
:10124300C622E4FFEFC39405748094805012EFC468
:1012530054F02401F582E43402F583E4F00F80E4D2
:1012630022AD07AC06E4F5C7ECF5C3EDF5C475C7CD
:101273008075C50175C65A75C6A500AFC22278240C
:10128300760008A607AE04AF05EE3395E08F0E8E09
:101293000DF50CF50B7F03020DEB4387807598501A
:1012A300538EFE53890F438920758BF3758DF3C2DB
:1012B300ABD28ED29922900330E0FF7E006401709E
:1012C30003309207EF4E700620930312000E0212B2
:1012D300D4209206E490032FF02290032F2093044E
:1012E3007402F0227401F0225389F0438901758C52
:1012F300F8758A30D2A9D28CE4F51DF51C22900230
:1013030000E004F075F00A84E5F0F0E07003C2B386
:0E13130022D2B32212772A264786823702069C
:00000001FF
